:100000007BC09EC09DC09CC09BC09FC099C098C033
:1000100097C096C095C094C093C092C091C07445DB
:1000200079467D47824887498B60906194629963E5
:100030009D64A265A766AB67B068B469B980BE81EC
:10004000C282C783CB84D084D484FF210000000007
:1000500000000000000000000000000000000000A0
:100060000000000000000000000000000000000090
:100070002167B1FF030405070A0E1319212B36432C
:1000800053657990AAC6E6FFFFFFFFFFFFFFFFFF62
:10009000FFFFFFFFFFFFFFFFFFFFFF00000000006B
:1000A0000000000000000000000000000000000050
:1000B00008121C2834414E5C6B7C8FA3B8CFE6FF3E
:1000C000FFFFFF0028000628000617280006111C65
:1000D0002800060E171F2800060C131A21280014EA
:1000E00028EA00EAF406142800EA060C131D28008A
:1000F00006132000F4EA280011241FBECFEDCDBF67
:1001000020E0A0E6B0E001C01D92A238B207E1F7FE
:10011000E1E6F0E085E5808781E083831482128246
:100120008683118288E081878FE48287612CECE6E8
:10013000F0E08DEF87838EEF8583712C98D09BC282
:100140005FCF1BBC19BC18BC0895189525B7277E36
:1001500025BF29B7226029BF21E022BF019728F0DF
:1001600020E188952150E9F7F9CF089588EE93E0D2
:10017000EDCF369A3699FECF85B10895CF93C72D2E
:1001800081E0870D8F73782E662D90E066D26FEF39
:100190008C2F90E0CF9161C2FF920F931F93CF936A
:1001A000DF93F82E0BE610E0C5E7D0E0F11005C0B4
:1001B000CE014BD2F801808304C0F8016081CE01EA
:1001C0004CD2219601501109CF37D10579F7DF9133
:1001D000CF911F910F91FF900895D0DF81E0DCCF88
:1001E000811101C0AECF815090E0FC01E45BFF4F74
:1001F000E491EBBDFC01EC58FF4FE491E9BDFC013B
:10020000E456FF4F849188BD08950F931F93CF93B9
:10021000C82F8B01CC2359F08AE0E2DFC80196DFBA
:1002200090DFC80193DFC80191DFC150F3CFCF91B8
:100230001F910F9108951F93CF93DF938FEA87B992
:1002400086EC86B910E1C0E0D0E085E090E07EDF8A
:1002500090DFC80FD11D1150C1F7CE0124E0969553
:1002600087952A95E1F7DF91CF911F9108951F920D
:10027000CDB7DD2783EA87B986EC86B93699FECFFC
:10028000369A3699FECF85B18095882E8FEF8DBD39
:1002900080E68CBD8FE384BB8BE187BB88EE88BB97
:1002A00081E083BF91EA9ABD80BF85B7806285BF38
:1002B000789487E790E0C9D1853511F08EDF11C0C1
:1002C000712C872D90E0C1D1682E8F3F19F080E00E
:1002D00063DF07C0872D91E0970D792E803488F376
:1002E000F6CF80916A001091640000916500F09053
:1002F0006200FF2019F000E010E089E08F5F90E0DD
:1003000040E050E064EC70E0882379F09B012F5FBF
:100310003F4FF9013197E491EE2319F0922F961B8C
:10032000F6CF8150AB01B901EFCF892F612F70E07B
:10033000A92FB0E0E82FF0E0002321F09D012E1B53
:100340003F0B05C09F0121503109260F371F319700
:10035000E40FF51FE4902B583F4FF901E0828150E4
:1003600049F7910F90936000112371F0002329F059
:10037000292F30E02150310902C020E030E0F9019E
:10038000EB58FF4F81E0808383E0890F282F2150B5
:10039000E22FE91BF0E0EC50FF4FE491A22FB0E018
:1003A000AB58BF4FEC932913F2CFE82FF0E0EC5895
:1003B000FF4F21E0409175003081431320E0821B04
:1003C000282F80938100862D853F78F5382D313494
:1003D00060F48F5F682E891708F0612C809182008D
:1003E0008F5F8F718093820020C0109282003F3A0D
:1003F000B0F430916700332311F0FF2031F08F5FAC
:10040000682E891790F0612C10C06916E1F3662000
:1004100019F08150682E09C02150622E06C0F110DB
:10042000F2CF80916300882371F3A8DE81EA87B957
:1004300086EC86B9C62CF4EFF61508F441C080911D
:100440008200803138F4E62DF0E0EB58FF4FB080A9
:10045000CB2C36C08BDE1092820052E6C52E50E0C7
:10046000D52E00E010E0FF24F39481E0800F0F5FB1
:100470001F4FF60190819F3F39F4FFEFCF1ADF0A3B
:100480000830110591F7DFCF6DE570E0BEDEF801B1
:10049000E459FF4F6080F60180818F2580839DDEC7
:1004A0006FE070E080E2B1DEF60180818F2580830D
:1004B00094DE612C5BDE809162008823F1F2C3CF71
:1004C00010E000E031EAE32E46ECD42EFAEECF1233
:1004D00016C021E0822F298383DE88E290E036DE99
:1004E00029812F5F2932B1F788E2F82E8F2D78DE2F
:1004F00088E290E02BDEFA94F110F8CF5DC084EF33
:10050000C8122AC084E690E021DE33DE90E0292F75
:1005100030E0F901E25EFF4FE491E81710F49E5FCE
:10052000F6CFF901E15EFF4FF4906DE770E08F2D9B
:1005300082958695877069DE8EEE92E007DE65E033
:1005400070E081E062DE85E694E000DE6DE770E059
:100550008F2D8F715ADE10C09EEFC91210C0612C12
:10056000F12CF0926A0039DE6AEF70E081E04DDE36
:10057000F394E9E0FE12F5CFF9DDF8DD1DC0FDEFE3
:10058000CF122AC0612C8FEF80936B0026DE8AE0A9
:1005900027DEECDDEBDD88E223DE4DDE80936B00B1
:1005A0001CDEE4DDE3DDF9CF0F5F0930F8F484EF02
:1005B00091E0CCDD10928200DCDD823808F043C08F
:1005C0001F5F183008F482CF98E29B1500F510E009
:1005D00094E1B92E24E1C22E8B2D02DE2CDEE7B889
:1005E000D6B820916B00281730F4DECF85E08B154C
:1005F000F0F6BA940AC090E030E022503109821738
:1006000093071CF4BC1408F4B39400E0D0CFE1E0ED
:10061000EB1530F48B2D86958695B694B80E12C0E6
:1006200090DD85B7877E806185BFF89485B7846843
:1006300085BF8B7F85BF85B7806285BF889585B76D
:100640008F7D85BFCB2C10E041CFE199FECF1FBA43
:100650008EBBE09A99278DB30895262FE199FECF9E
:100660001CBA1FBA8EBB2DBB0FB6F894E29AE19A62
:0A0670000FBE01960895F894FFCF25
:00000001FF
